:020000040000FA
:020000000528D1
:040002000034003492
:080008000528BF22E122772048
:100010006720772038107F20AA2006130D210C2896
:1000200082074634723465347134753465346E3405
:100030006334793443346F3475346E3474346534D6
:100040007234A2345034493443342D34463443346A
:10005000A3345634653472342E3431342E34303473
:10006000313482072E3430343134733420342E341A
:100070003134733420342034313473342034313407
:1000800030347334820741346D3470342E3450343C
:100090002E3453342E3443346834313420344334D2
:1000A0006834323420348207003410341834183461
:1000B0001C341C341E341F341030B10006163208B4
:1000C0001020B3003B23B20AB10B5F280800B20135
:1000D0005C200612C030B3003B235C20B501EB234B
:1000E000B501EB23B501EB23B501EB2308000612A4
:1000F0000130B3003B230230B500EB2308000612A9
:100100008030B3003B2306162308B100B10DB10DBA
:100110000C30B10531084220B3003B23B10A31084D
:100120004220B3003B23B10A31084220B3003B23F5
:10013000B10A31084220B3003B23B10A0612CC3089
:10014000B3003B232208B200B20DB20D0C30B20551
:10015000022108000612C030B3003B23B401381B53
:10016000B411381FB4158330B40434089F00061648
:10017000B301381F3310381B33144130B3073B230E
:1001800083169F0183121F151F19C4281E08A4007F
:10019000831607309F0083120310A40C0310A40CD5
:1001A0000830B2000730B300083024020318DF28FB
:1001B00006162408B3003B23B301A401E128061668
:1001C0003B230830A402B20BD428A501A601A70145
:1001D000A801A9011E08A4009A210830840700087C
:1001E000B3003030B3073B23840A0008B30030303B
:1001F000B3073B23840A0008B3003030B3073B2326
:10020000840A08000430B100061632083120B30019
:100210003B23B20AB10B05290800A401A501A601E0
:10022000A701A801A90106128430B3003B230616DA
:100230002308B400B409B40DB41CB411B418B41537
:100240003416340885008A018A0A22080339820795
:10025000832B8B2B8F2B932B0800362136213621B5
:100260003621362136213621362136213F213F21C4
:100270003F213F213F213F213F213F213F21482175
:100280004821482148214821482148214821482126
:10029000FD2154215E215321532153215321532108
:1002A0005321532153215C215C215C215C215C2181
:1002B0005C215C215C215C21652165216521652132
:1002C000652165216521652165210108A0002008BF
:1002D000A102A109A10A2108A40701300318A5075A
:1002E0000318A6070318A7070318A8070318A907E8
:1002F0002008A10008000108A10000000000000083
:1003000000000000000000000000000000000000ED
:1003100000000000000000000000000000000000DD
:10032000080092210310A40DA50DA60DA70DA80D80
:10033000A90D080070308400A821A821A821A821B7
:10034000A821A821A821A821A821A821A821080026
:100350003030B500AB01AC01AD01AE01AF01B00171
:10036000AA010310A40DA50DA60DA70DA80DA90D9A
:10037000AA0D0A302A02031CC1290A30AA0203145A
:10038000C2290310AB0DAC0DAD0DAE0DAF0DB00D10
:10039000B50BB1292B08A4002C08A5002D08A60038
:1003A0002E08A7002F08A8003008A90084032A08F7
:1003B000800008000616003032020319E929703067
:1003C0000402031CE9297830B300840AB10A3B23F4
:1003D00008000008B300840A00303102031DF4292C
:1003E000003033020319F929B10A3030B3073B2337
:1003F00008002030B3003B2308005F3066008316FE
:100400008113831200000000000000000608B40001
:10041000B409831681178312003066003408B600D1
:10042000361EB610361AB6140330B6053408B706B1
:100430003408B705B81B2C2AB7187B2A37199A2A13
:10044000371BAE2AB7193B2A3408B700000000005A
:100450000000000000000800B718752A37198F2A1D
:10046000B719352A3408B70008003408B7003F3000
:10047000B80577200A283408B7004030B807B81FFD
:100480000A2838107720061706128030B3003B2365
:1004900006164130B3003B238B309F000530B5007A
:1004A000EB23C0200612C030B3003B2306164230B7
:1004B000B3003B2383309F000530B500EB23C02001
:1004C0002208B200B20DB20D0C30B20502210613A3
:1004D00002308A002208220782074821432A3F214E
:1004E000432A3621432A2D21432A3408B700A20A81
:1004F0000330A205412A3408B700A20A0330A2053E
:100500000A2806164830B3003B234F30B3003B2384
:100510004C30B3003B234430B3003B230800340885
:10052000B7003818412A381406128C30B3003B2328
:100530008122A42A3408B70038180A283814061271
:100540008030B3003B2381220A30B500EB23FD212C
:10055000A42A8207E834E034E134E2343408B700F6
:10056000A30A0330A30502308A002308A9228101CF
:1005700064008316810007309F0083120A28A301BC
:10058000A201B801B701B601133065001330850030
:1005900086010F30660000000608B700B70900307A
:1005A00066000313831607309F00E8308100831232
:1005B0000130A2000330A3008316E23081008312D1
:1005C000080006120F30B500EB2309308600202307
:1005D0000530B500EB230930860020236430B500D8
:1005E0000124093086002023013086002023283092
:1005F000B3003B230130B3003B230230B500EB23B3
:100600000630B3003B230C30B3003B234030B30033
:100610003B230616B1010730B20031085320B30066
:100620003B23B20B0D2B1F30B3003B23B10A310823
:10063000073C03180B2B06128030B3003B23080045
:100640000000000086160000000086123C30B50055
:1006500001240800820700340834013409340434CA
:100660000C3405340D3402340A3403340B340634AC
:100670000E3407340F3403308A003308B400B40E4C
:100680000F30B40534082A23B400061F3413061BA8
:100690003417061E3412061A341634088600202336
:1006A0003308B4000F30B40534082A23B400061F01
:1006B0003413061B3417061E3412061A3416340877
:1006C000860020238A01080003308A00230882075D
:1006D0007E2B6C2B7D2B7C2B03308A003608820707
:1006E0009221922192219221922191219121912175
:1006F00006179A21B20108009221912106179A212A
:100700000130B20008007B2148216423840A840A56
:10071000840A972308007B213F216423872B7B21B8
:1007200036216423882B7B212D216423892BB10161
:10073000023000020318B82BDA21DA21DA21003066
:100740003102031DC72BE623DA21DA21DA2100303A
:100750003102031DD32BDA21DA21DA21B10ADA21A1
:100760002E30B3003B23DA212030B3003B23DF2BB4
:10077000DA212E30B3003B23DA21DA21DA21DA2123
:10078000DA21DA21DA214730B3003B23DF2BDA21EB
:100790002E30B3003B23DA21DA21DA21DA214D3081
:1007A000B3003B23DF2BDA212E30B3003B23DA21C9
:1007B000DA21DA21DA214B30B3003B23DF2B48303A
:1007C000B3003B237A30B3003B2308000612843089
:1007D000B3003B230800B601000000000000000049
:1007E0000000000000000000000000000000000009
:1007F0000000000000000000B60BEC2BB50BEB2B4B
:0E0800000800000000000000B50B012C0800ED
:02400E00B23FBF
:00000001FF
